:020000040000FA
:10000000831603131F308500860187018E309F0001
:1000100003178C130313831241309F00850186015F
:10002000870103178D0183160C1483120C08A60098
:100030008D0A83160C1483120C08A70003133830A2
:10004000C2200230E5200630C2200230E5200C300C
:10005000C2200230E5200130C2200230E520A50197
:1000600025086E20C420A50A2508103C031D302851
:10007000C030C2200130E520A50125087F20C42022
:10008000A50A2508103C031D3D28F32000211F155B
:100090001F19482883161E088312A80003101E1873
:1000A0000314A80C2608013E2802031C0716270883
:1000B0002802031807122808CF208D30C2202208FA
:1000C000C4202108C4202008C420851C9020051DC0
:1000D0009520851DA020051EA520472882075434A1
:1000E00045344D345034453452344134543455340D
:1000F000523441343A3420342034203420348207BE
:100100002034203420342034203420347F342D34E3
:100110002D347E34203420342034203420342034D4
:10012000A60AF320851C92289928A603F320051D12
:10013000972803178D0126088C00B1200313BD28D2
:10014000A70A0021851DA228A928A7030021051EB2
:10015000A728031701308D0027088C00B120031356
:10016000BD2883160C1555308D00AA308D008C14D7
:100170000C118C18B9288312080087156430E5200B
:10018000871108008713C528871786000130E520EE
:1001900007170130E52007130130E5200800A00013
:1001A000A101A2016430A002031CD828A20AD3280E
:1001B000A0070A30A002031CDF28A10ADA28A00742
:1001C0003030A007A107A2070800A4006E30A300EA
:1001D000000000000000000000000000A30BE82861
:1001E000A40BE62808002608CF20C230C220013028
:1001F000E5202208C4202108C4202008C4200800CB
:100200002708CF20CB30C2200130E5202208C420AF
:0A0210002108C4202008C4200800C3
:044200002800320060
:00000001FF
